:100000000C9438000C9453000C9453000C9453003F
:100010000C9453000C9453000C9453000C94530014
:100020000C9453000C9453000C9453000C94530004
:100030000C9453000C9453000C9453000C945300F4
:100040000C9453000C94C1020C9453000C94530074
:100050000C94980F0C9453000C9453000C94530080
:100060000C9453000C9453000C9453000C945300C4
:1000700011241FBECFEFD4E0DEBFCDBF13E0A0E060
:10008000B1E0E4E2F4E202C005900D92AC3BB107AE
:10009000D9F714E0ACEBB3E001C01D92A93AB10767
:1000A000E1F70C9472000C940000CF93DF93CDB76E
:1000B000DEB7E4E3F0E08FEF8083EAE3F0E08EE286
:1000C0008083ABE3B0E0EBE3F0E0808182608C936F
:1000D000ABE3B0E0EBE3F0E0808180628C93DF91F2
:1000E000CF910895CF93DF93CDB7DEB70E9455002F
:1000F0000E94B2020E94960E7894A5E3B0E0E5E378
:10010000F0E0808181608C930E9485020E94FD0254
:100110000E9447030E9491030E94DB030E94250472
:100120000E946F040E94B9040E9403050E944D05BD
:100130000E9497050E940C0700C08091BE03813089
:1001400031F41092BE030E9478110E9487118091B1
:10015000CB038130E1F4A5E3B0E0E5E3F0E080819A
:1001600084608C930E94A20D0E942A100E94AC070A
:100170000E94C1080E94F5090E9458060E943D078E
:10018000A5E3B0E0E5E3F0E080818B7F8C93809184
:10019000BC03813091F61092BC030E94E105CDCFE3
:1001A000CF93DF93CDB7DEB764E084E00E94ED002B
:1001B0006CE480E00E94ED001092BE038091BE03CB
:1001C0008823E1F36AE08CE60E94ED0060E085E0C0
:1001D0000E94ED00DF91CF910895CF93DF93CDB7CB
:1001E000DEB724970FB6F894DEBF0FBECDBF8B836A
:1001F0006C83ABE3B0E0EBE3F0E080818D7F8C9328
:1002000087E08A8340C0ABE3B0E0EBE3F0E08081BD
:10021000877F8C9300000000000000008A81282F57
:10022000332727FD309581E090E0022E02C0880F31
:10023000991F0A94E2F7982F8B81892389838981FA
:10024000882341F0ABE3B0E0EBE3F0E08081846031
:100250008C9307C0ABE3B0E0EBE3F0E080818B7FF1
:100260008C930000000000000000ABE3B0E0EBE383
:10027000F0E0808188608C930000000000000000A6
:100280008A8181508A838A8188230CF0BCCF87E0E1
:100290008A8340C0ABE3B0E0EBE3F0E08081877F8E
:1002A0008C9300000000000000008A81282F332773
:1002B00027FD309581E090E0022E02C0880F991F43
:1002C0000A94E2F7982F8C81892389838981882376
:1002D00041F0ABE3B0E0EBE3F0E0808184608C932D
:1002E00007C0ABE3B0E0EBE3F0E080818B7F8C9361
:1002F0000000000000000000ABE3B0E0EBE3F0E042
:10030000808188608C9300000000000000008A81DA
:1003100081508A838A8188230CF0BCCFABE3B0E0A4
:10032000EBE3F0E08081877F8C93ABE3B0E0EBE31D
:10033000F0E080818B7F8C93ABE3B0E0EBE3F0E007
:10034000808182608C9324960FB6F894DEBF0FBE36
:10035000CDBFDF91CF910895CF93DF93CDB7DEB7B7
:1003600024970FB6F894DEBF0FBECDBF8C83ABE3EE
:10037000B0E0EBE3F0E080818D7F8C9387E08A83AF
:100380004CC0ABE3B0E0EBE3F0E08081877F8C937F
:10039000000000000000000000000000000000005D
:1003A0008A81282F332727FD309581E090E0022EA7
:1003B00002C0880F991F0A94E2F7982F8C81892335
:1003C0008B838B81181644F4ABE3B0E0EBE3F0E0F1
:1003D000808184608C9307C0ABE3B0E0EBE3F0E096
:1003E00080818B7F8C9300000000000000000000E3
:1003F000000000000000ABE3B0E0EBE3F0E0808140
:1004000088608C93000000000000000000000000E5
:10041000000000008A8181508A838A8188230CF041
:10042000B0CF1B82ABE3B0E0EBE3F0E08081877FED
:100430008C9300000000000000000000000000009D
:10044000000087E08A833DC0ABE3B0E0EBE3F0E07F
:10045000808188608C93E9E3F0E0808189838981E1
:10046000992780719070181619068CF48A81282FAC
:10047000332727FD309581E090E0022E02C0880FDF
:10048000991F0A94E2F7982F8B81892B8B830000A8
:100490000000000000000000000000000000ABE3CE
:1004A000B0E0EBE3F0E08081877F8C9300000000F8
:1004B0000000000000000000000000008A81815060
:1004C0008A838A8188230CF0BFCFABE3B0E0EBE3F3
:1004D000F0E08081877F8C93ABE3B0E0EBE3F0E06A
:1004E00080818B7F8C93ABE3B0E0EBE3F0E0808125
:1004F00082608C938B81992724960FB6F894DEBF87
:100500000FBECDBFDF91CF910895CF93DF93CDB7CD
:10051000DEB70E94D0001092BC038091BC038823F8
:10052000E1F30E941E060E94C70B1092BC0380914B
:10053000BC038823E1F31092BC038091BC038823A1
:10054000E1F31092BC0364E084E00E94ED006CE4EF
:1005500080E00E94ED000E94E1050E947706DF9195
:10056000CF910895CF93DF93CDB7DEB7E3E5F0E009
:1005700082E08083E9E5F0E082E08083DF91CF9143
:1005800008951F920F920FB60F9211248F93CF935D
:10059000DF93CDB7DEB78091C0038F5F8093C00338
:1005A0008091C003883409F581E08093BF031092E5
:1005B000C003809164048F5F80936404809164041D
:1005C000843629F41092640481E08093BC03809106
:1005D00063048F5F80936304809163048A3029F4FD
:1005E0001092630481E08093BE03DF91CF918F91DD
:1005F0000F900FBE0F901F901895CF93DF93CDB73C
:10060000DEB762E480E00E94ED001092BC038091AE
:10061000BC038823E1F31092BC0364EA89E00E94E2
:10062000ED001092BE038091BE038823E1F3109287
:10063000BE031092650416C080916504682F8AE09D
:100640000E94ED00809165049927FC01E95CFE4F52
:100650008081682F8BE00E94ED00809165048F5FA0
:100660008093650480916504863330F360EA88E006
:100670000E94ED001092BE038091BE038823E1F337
:100680006CE480E00E94ED00DF91CF910895CF935C
:10069000DF93CDB7DEB762E480E00E94ED001092F8
:1006A000BC038091BC038823E1F31092BC0365EA8C
:1006B00089E00E94ED001092BE038091BE03882362
:1006C000E1F31092BE031092650416C08091650498
:1006D000682F8AE00E94ED00809165049927FC0153
:1006E000E958FE4F8081682F8BE00E94ED008091D9
:1006F00065048F5F8093650480916504863330F3D1
:1007000060EA88E00E94ED001092BE038091BE0373
:100710008823E1F36CE480E00E94ED00DF91CF914B
:100720000895CF93DF93CDB7DEB762E480E00E94F7
:10073000ED001092BC038091BC038823E1F310927A
:10074000BC0366EA89E00E94ED001092BE0380912E
:10075000BE038823E1F31092BE031092650416C015
:1007600080916504682F8AE00E94ED008091650405
:100770009927FC01E954FE4F8081682F8BE00E948D
:10078000ED00809165048F5F80936504809165041E
:10079000863330F360EA88E00E94ED001092BE03D9
:1007A0008091BE038823E1F36CE480E00E94ED00B9
:1007B000DF91CF910895CF93DF93CDB7DEB762E499
:1007C00080E00E94ED001092BC038091BC0388235E
:1007D000E1F31092BC0367EA89E00E94ED001092F9
:1007E000BE038091BE038823E1F31092BE031092F2
:1007F000650416C080916504682F8AE00E94ED00B0
:10080000809165049927FC01E950FE4F8081682F93
:100810008BE00E94ED00809165048F5F80936504FA
:1008200080916504863330F360EA88E00E94ED0031
:100830001092BE038091BE038823E1F36CE480E054
:100840000E94ED00DF91CF910895CF93DF93CDB754
:10085000DEB762E480E00E94ED001092BC0380915C
:10086000BC038823E1F31092BC0368EA89E00E948C
:10087000ED001092BE038091BE038823E1F3109235
:10088000BE031092650416C080916504682F8AE04B
:100890000E94ED00809165049927FC01E95CFD4F01
:1008A0008081682F8BE00E94ED00809165048F5F4E
:1008B0008093650480916504863330F360EA88E0B4
:1008C0000E94ED001092BE038091BE038823E1F3E5
:1008D0006CE480E00E94ED00DF91CF910895CF930A
:1008E000DF93CDB7DEB762E480E00E94ED001092A6
:1008F000BC038091BC038823E1F31092BC0369EA36
:1009000089E00E94ED001092BE038091BE0388230F
:10091000E1F31092BE031092650416C08091650445
:10092000682F8AE00E94ED00809165049927FC0100
:10093000E958FD4F8081682F8BE00E94ED00809187
:1009400065048F5F8093650480916504863330F37E
:1009500060EA88E00E94ED001092BE038091BE0321
:100960008823E1F36CE480E00E94ED00DF91CF91F9
:100970000895CF93DF93CDB7DEB762E480E00E94A5
:10098000ED001092BC038091BC038823E1F3109228
:10099000BC036AEA89E00E94ED001092BE038091D8
:1009A000BE038823E1F31092BE031092650416C0C3
:1009B00080916504682F8AE00E94ED0080916504B3
:1009C0009927FC01E954FD4F8081682F8BE00E943C
:1009D000ED00809165048F5F8093650480916504CC
:1009E000863330F360EA88E00E94ED001092BE0387
:1009F0008091BE038823E1F36CE480E00E94ED0067
:100A0000DF91CF910895CF93DF93CDB7DEB762E446
:100A100080E00E94ED001092BC038091BC0388230B
:100A2000E1F31092BC036BEA89E00E94ED001092A2
:100A3000BE038091BE038823E1F31092BE0310929F
:100A4000650416C080916504682F8AE00E94ED005D
:100A5000809165049927FC01E950FD4F8081682F42
:100A60008BE00E94ED00809165048F5F80936504A8
:100A700080916504863330F360EA88E00E94ED00DF
:100A80001092BE038091BE038823E1F36CE480E002
:100A90000E94ED00DF91CF910895CF93DF93CDB702
:100AA000DEB762E480E00E94ED001092BC0380910A
:100AB000BC038823E1F31092BC036CEA89E00E9436
:100AC000ED001092BE038091BE038823E1F31092E3
:100AD000BE031092650416C080916504682F8AE0F9
:100AE0000E94ED00809165049927FC01E95CFC4FB0
:100AF0008081682F8BE00E94ED00809165048F5FFC
:100B00008093650480916504863330F360EA88E061
:100B10000E94ED001092BE038091BE038823E1F392
:100B20006CE480E00E94ED00DF91CF910895CF93B7
:100B3000DF93CDB7DEB762E480E00E94ED00109253
:100B4000BC038091BC038823E1F31092BC036DEADF
:100B500089E00E94ED001092BE038091BE038823BD
:100B6000E1F31092BE031092650416C080916504F3
:100B7000682F8AE00E94ED00809165049927FC01AE
:100B8000E958FC4F8081682F8BE00E94ED00809136
:100B900065048F5F8093650480916504863330F32C
:100BA00060EA88E00E94ED001092BE038091BE03CF
:100BB0008823E1F36CE480E00E94ED00DF91CF91A7
:100BC0000895CF93DF93CDB7DEB789ED80936504A9
:100BD00013C060E085E00E94ED0080916504682FFD
:100BE00086E00E94ED0064E587E00E94ED008091C0
:100BF00065048F5F80936504809165048C3D48F3A4
:100C000085EE8093650413C060E085E00E94ED00EE
:100C100080916504682F86E00E94ED0064E587E01E
:100C20000E94ED00809165048F5F80936504809140
:100C30006504883E48F3DF91CF910895CF93DF9309
:100C4000CDB7DEB764970FB6F894DEBF0FBECDBF49
:100C50008DE589838EE58A838FE58B8389E48C8398
:100C60008BE58D838DE18E838CE58F83188680E202
:100C7000898789E28A8786E38B8781E48C878AE08B
:100C80008D8781E48E8781E08F8786E2888B20E1E3
:100C9000CE010196AC0162E087E00E94A206649654
:100CA0000FB6F894DEBF0FBECDBFDF91CF91089590
:100CB000CF93DF93CDB7DEB760E085E00E94ED0013
:100CC0006FEC86E00E94ED006CE887E00E94ED008A
:100CD00061E085E00E94ED006BE086E00E94ED009F
:100CE0006DE887E00E94ED00DF91CF910895CF93EA
:100CF000DF93CDB7DEB760E085E00E94ED0060E2F3
:100D000086E00E94ED0060E887E00E94ED0060E070
:100D100085E00E94ED006EE386E00E94ED0064E84D
:100D200087E00E94ED0060E085E00E94ED006CE548
:100D300086E00E94ED0068E887E00E94ED00DF9108
:100D4000CF910895CF93DF93CDB7DEB72D970FB630
:100D5000F894DEBF0FBECDBF89876A875C874B875B
:100D60002D878A85282F33278EE190E0A901489F9F
:100D70009001499F300D589F300D11248985992786
:100D8000820F931F98878F838D85282F33278F811C
:100D90009885820F931F9E838D83109265048F81A7
:100DA00098859C838B8328C08B818A838B819C81CF
:100DB000892F99278983698185E00E94ED006A81E6
:100DC00086E00E94ED0040916504842F99279C01E4
:100DD0008B859C85F901E80FF91F8081982F842F5E
:100DE0008F5F80936504692F87E00E94ED008B81FF
:100DF0009C8101969C838B832B813C818D819E817C
:100E00002817390788F22D960FB6F894DEBF0FBE6B
:100E1000CDBFDF91CF910895CF93DF93CDB7DEB7EC
:100E200081E091E029E0AC016EE083E00E94A2063F
:100E3000DF91CF910895CF93DF93CDB7DEB722979F
:100E40000FB6F894DEBF0FBECDBF8A838A81882398
:100E500021F48A818652898303C08A8180538983E1
:100E60008981992787FD909522960FB6F894DEBF69
:100E70000FBECDBFDF91CF9108950F931F93CF93F6
:100E8000DF93CDB7DEB72D970FB6F894DEBF0FBE58
:100E9000CDBF80917204909173042EE130E0B901CE
:100EA0000E94EB11CB019B838A83CE0104962A8199
:100EB0003B814AE050E0BC01C9010E94BA11CE0159
:100EC0000496DC01FD0101900020E9F73197CF0184
:100ED0008A1B9B0B8983109265041CC0809165045A
:100EE000082F112780916504282F3327CE010496FF
:100EF000FC01E20FF31F80810E941B07282FCE0107
:100F00000996FC01E00FF11F2083809165048F5F3B
:100F10008093650480916504282F33278981992760
:100F200087FD909528173907CCF2298199818BE0AC
:100F3000382F391BCE010996AC016EE0832F0E9439
:100F4000A2062D960FB6F894DEBF0FBECDBFDF917F
:100F5000CF911F910F910895CF93DF93CDB7DEB757
:100F600029970FB6F894DEBF0FBECDBF80917A04EB
:100F700090917B048E5590409C838B838B819C81C8
:100F800023E030E0B9010E94EB11CB019A83898301
:100F900089819A818A30910524F089E090E09A83D2
:100FA000898389819A81992314F41A821982209164
:100FB000C4033091C50389819A818217930709F48C
:100FC000D7C089819A81823091052CF460E184E058
:100FD0000E94ED0004C060E084E00E94ED00898181
:100FE0009A819093C5038093C40380E88D8384E83D
:100FF0008E8388E88F8389819A81998788878885FD
:1010000099858430910509F45FC08885998585307C
:101010009105DCF4888599858130910509F43FC0FC
:1010200088859985823091052CF48885998500976B
:1010300079F173C08885998582309105B9F18885E9
:10104000998583309105C9F168C088859985873075
:10105000910509F44EC088859985883091055CF426
:101060008885998585309105B1F188859985863087
:101070009105C1F152C0888599858830910509F4A0
:101080003FC0888599858930910509F440C045C0E5
:1010900080E88D8384E88E8388E88F833EC081E872
:1010A0008D8384E88E8388E88F8337C082E88D83C0
:1010B00084E88E8388E88F8330C083E88D8384E85A
:1010C0008E8388E88F8329C083E88D8385E88E83AB
:1010D00088E88F8322C083E88D8386E88E8388E842
:1010E0008F831BC083E88D8387E88E8388E88F8396
:1010F00014C083E88D8387E88E8389E88F830DC0D1
:1011000083E88D8387E88E838AE88F8306C083E82F
:101110008D8387E88E838BE88F8360E085E00E9473
:10112000ED0060E286E00E94ED008D81682F87E08F
:101130000E94ED0060E085E00E94ED006EE386E035
:101140000E94ED008E81682F87E00E94ED0060E034
:1011500085E00E94ED006CE586E00E94ED008F8145
:10116000682F87E00E94ED0060E084E00E94ED00BF
:1011700029960FB6F894DEBF0FBECDBFDF91CF9199
:101180000895CF93DF93CDB7DEB726970FB6F894C7
:10119000DEBF0FBECDBF80916A0490916B0426E143
:1011A00030E0B9010E94EB11CB0106969E838D833E
:1011B0008D819E8199230CF446C08D819E812AE009
:1011C00030E0B9010E94EB11CB018A838D819E81B1
:1011D0002AE030E0B9010E94EB118983898186956C
:1011E0008C5F89838A81282F332786E890E0821BD1
:1011F000930B9C838B8320910D0130910E018B8189
:101200009C818217930761F080910D0190910E01EE
:101210000E947A098B819C8169810E94B4090AC06D
:101220009091C9038981981729F08B819C816981EC
:101230000E94B40989818093C9038B819C8190931A
:101240000E0180930D018D819E8199230CF049C080
:101250008D819E81909581959F4F9E838D838D81F9
:101260009E812AE030E0B9010E94EB11CB018A8314
:101270008D819E812AE030E0B9010E94EB118983C3
:101280008981869589838A8199278A579F4F9C8374
:101290008B8320910D0130910E018B819C818217EF
:1012A000930761F080910D0190910E010E947A09DF
:1012B0008B819C8169810E94B4090AC09091C90305
:1012C0008981981729F08B819C8169810E94B409DA
:1012D00089818093C9038B819C8190930E018093B7
:1012E0000D0126960FB6F894DEBF0FBECDBFDF917D
:1012F000CF910895CF93DF93CDB7DEB726970FB682
:10130000F894DEBF0FBECDBF9E838D831C821B82EF
:101310001DC08D818A838D819E81892F9927898324
:10132000698185E00E94ED006A8186E00E94ED00FF
:1013300060E087E00E94ED008D819E814E969E8345
:101340008D838B819C8101969C838B838B819C8177
:1013500088309105F0F226960FB6F894DEBF0FBEE6
:10136000CDBFDF91CF910895CF93DF93CDB7DEB797
:1013700027970FB6F894DEBF0FBECDBF9E838D8337
:101380006F831C821B8223C08D818A838D819E8105
:10139000892F99278983698185E00E94ED006A8100
:1013A00086E00E94ED008F819927FC01E35DFE4FEE
:1013B0008081682F87E00E94ED008D819E814E968E
:1013C0009E838D838B819C8101969C838B838B81F3
:1013D0009C8188309105C0F227960FB6F894DEBF45
:1013E0000FBECDBFDF91CF910895CF93DF93CDB7DF
:1013F000DEB726970FB6F894DEBF0FBECDBF809143
:1014000068049091690426E130E0B9010E94EB1173
:10141000CB019E838D838D819E8199230CF452C0D4
:101420008D819E812AE030E0B9010E94EB11CB0151
:101430008A838D819E812AE030E0B9010E94EB1100
:1014400089838981869589838A81282F332787E03C
:1014500090E0AC01421B530B9A018EE190E0AC018D
:10146000249FC001259F900D349F900D11240A9652
:101470009C838B8320910B0130910C018B819C818B
:101480008217930761F080910B0190910C010E94EB
:10149000C50A8B819C8169810E94280B0AC09091AA
:1014A000C8038981981729F08B819C8169810E94EA
:1014B000280B89818093C8038B819C8190930C01B8
:1014C00080930B018D819E8199230CF055C08D81F5
:1014D0009E81909581959F4F9E838D838D819E8166
:1014E0002AE030E0B9010E94EB11CB018A838D81A3
:1014F0009E812AE030E0B9010E94EB118983898145
:1015000086958C5F89838A81282F33278EE190E02E
:10151000AC01249FC001259F900D349F900D112494
:1015200086509F4F9C838B8320910B0130910C013F
:101530008B819C818217930761F080910B019091C0
:101540000C010E94C50A8B819C8169810E94280B35
:101550000AC09091C8038981981729F08B819C81DA
:1015600069810E94280B89818093C8038B819C81AB
:1015700090930C0180930B0126960FB6F894DEBF72
:101580000FBECDBFDF91CF910895CF93DF93CDB73D
:10159000DEB726970FB6F894DEBF0FBECDBF9E8391
:1015A0008D838D819E819C838B8318C08B818A83E0
:1015B0008B819C81892F99278983698185E00E948D
:1015C000ED006A8186E00E94ED0060E087E00E9405
:1015D000ED008B819C8101969C838B838D819E8104
:1015E0009C01275F3F4F8B819C8182179307F0F20C
:1015F0008091C803282F3327C901880F991F820FB4
:10160000931FFC01EF5EFE4F80818823C1F08D8126
:101610009E8182969C838B838B818A838B819C8124
:10162000892F99278983698185E00E94ED006A816D
:1016300086E00E94ED0060E087E00E94ED002696C3
:101640000FB6F894DEBF0FBECDBFDF91CF910895E6
:10165000CF93DF93CDB7DEB727970FB6F894DEBFF1
:101660000FBECDBF9E838D836F838D819E819C83B2
:101670008B8324C08B8189838B819C81892F9927BF
:101680008A836A8185E00E94ED00698186E00E947C
:10169000ED008F81282F3327C901880F991F820FF2
:1016A000931FFC01E15FFE4F8081682F87E00E945D
:1016B000ED008B819C8101969C838B838D819E8123
:1016C0009C01275F3F4F8B819C818217930790F28B
:1016D0008D819E8104969C838B838B8189838B81F2
:1016E0009C81892F99278A836A8185E00E94ED0079
:1016F000698186E00E94ED008F81282F3327C90180
:10170000880F991F820F931FFC01E05FFE4F8081BD
:10171000682F87E00E94ED008F81282F3327C901B1
:10172000880F991F820F931FFC01EF5EFE4F80818F
:10173000882321F18D819E8182969C838B838B816E
:1017400089838B819C81892F99278A836A8185E08F
:101750000E94ED00698186E00E94ED008F81282FB4
:101760003327C901880F991F820F931FFC01EF5E79
:10177000FE4F8081682F87E00E94ED0027960FB60C
:10178000F894DEBF0FBECDBFDF91CF910895CF9308
:10179000DF93CDB7DEB760E085E00E94ED0063E83F
:1017A00086E00E94ED0060E987E00E94ED0060E0C5
:1017B00085E00E94ED0064E886E00E94ED0061E9AA
:1017C00087E00E94ED0060E085E00E94ED0065E8A2
:1017D00086E00E94ED0062E987E00E94ED0060E093
:1017E00085E00E94ED0066E886E00E94ED0063E976
:1017F00087E00E94ED0060E085E00E94ED0067E870
:1018000086E00E94ED0064E987E00E94ED0060E060
:1018100085E00E94ED0068E886E00E94ED0065E941
:1018200087E00E94ED0060E085E00E94ED0069E83D
:1018300086E00E94ED0066E987E00E94ED0060E02E
:1018400085E00E94ED006AE886E00E94ED0067E90D
:1018500087E00E94ED0060E085E00E94ED0061EA13
:1018600086E00E94ED0068E987E00E94ED0060E0FC
:1018700085E00E94ED0062EA86E00E94ED0069E9E1
:1018800087E00E94ED0060E085E00E94ED0063EAE1
:1018900086E00E94ED006AE987E00E94ED0060E0CA
:1018A00085E00E94ED0064EA86E00E94ED006BE9AD
:1018B00087E00E94ED0060E085E00E94ED0065EAAF
:1018C00086E00E94ED006CE987E00E94ED0060E098
:1018D00085E00E94ED0066EA86E00E94ED006DE979
:1018E00087E00E94ED0060E085E00E94ED0067EA7D
:1018F00086E00E94ED006EE987E00E94ED0060E066
:1019000085E00E94ED0068EA86E00E94ED006FE944
:1019100087E00E94ED0060E085E00E94ED006FEB43
:1019200086E00E94ED0060EA87E00E94ED0060E042
:1019300085E00E94ED0060EC86E00E94ED0061EA27
:1019400087E00E94ED0060E085E00E94ED0061EC20
:1019500086E00E94ED0062EA87E00E94ED0060E010
:1019600085E00E94ED0062EC86E00E94ED0063EAF3
:1019700087E00E94ED0060E085E00E94ED0063ECEE
:1019800086E00E94ED0064EA87E00E94ED0060E0DE
:1019900085E00E94ED0064EC86E00E94ED0065EABF
:1019A00087E00E94ED0060E085E00E94ED0065ECBC
:1019B00086E00E94ED0066EA87E00E94ED0060E0AC
:1019C00085E00E94ED0066EC86E00E94ED0067EA8B
:1019D00087E00E94ED0060E085E00E94ED006DED83
:1019E00086E00E94ED0068EA87E00E94ED0060E07A
:1019F00085E00E94ED006EED86E00E94ED0069EA50
:101A000087E00E94ED0060E085E00E94ED006FED50
:101A100086E00E94ED006AEA87E00E94ED0060E047
:101A200085E00E94ED0060EE86E00E94ED006BEA2A
:101A300087E00E94ED0060E085E00E94ED0061EE2D
:101A400086E00E94ED006CEA87E00E94ED0060E015
:101A500085E00E94ED0062EE86E00E94ED006DEAF6
:101A600087E00E94ED0060E085E00E94ED0063EEFB
:101A700086E00E94ED006EEA87E00E94ED0060E0E3
:101A800085E00E94ED0064EE86E00E94ED006FEAC2
:101A900087E00E94ED0060E085E00E94ED006BEFC2
:101AA00086E00E94ED0060EB87E00E94ED0060E0C0
:101AB00085E00E94ED006CEF86E00E94ED0061EB96
:101AC00087E00E94ED0060E085E00E94ED006DEF90
:101AD00086E00E94ED0062EB87E00E94ED0060E08E
:101AE00085E00E94ED006EEF86E00E94ED0063EB62
:101AF00087E00E94ED0060E085E00E94ED006FEF5E
:101B000086E00E94ED0064EB87E00E94ED0061E05A
:101B100085E00E94ED0060E086E00E94ED0065EB4C
:101B200087E00E94ED0061E085E00E94ED0061E049
:101B300086E00E94ED0066EB87E00E94ED00DF91F9
:101B4000CF910895CF93DF93CDB7DEB764970FB6EB
:101B5000F894DEBF0FBECDBF83E090E09C8B8B8BF3
:101B60001A82198283E990E09C838B831092CB03C5
:101B7000CFC08B899C89FC01E453FC4F808199275D
:101B8000CD979A8B898B8B899C8901969C8B8B8BAB
:101B90008B899C89FC01E453FC4F80819927CD9768
:101BA000988B8F878B899C8901969C8B8B8B8B89DB
:101BB0009C89FC01E453FC4F80819927CD979E8737
:101BC0008D878B899C8901969C8B8B8B8B899C89BB
:101BD000FC01E453FC4F80819927CD979C878B872C
:101BE0008B899C8901969C8B8B8B89899A899C0116
:101BF000220F331F220F331F8F8598899595879564
:101C0000959587959595879595958795822B932B97
:101C10009A8789878F8598898F7090709C0122950B
:101C20003295307F3227207F32278D859E8595958E
:101C3000879595958795822B932B98878F838D8594
:101C40009E85837090709C0100243695279507949B
:101C5000369527950794322F202D8B859C85822BD6
:101C6000932B9E838D838B819C8101979C838B8397
:101C70008B819C812FEF8F3F920709F44EC08981A1
:101C80009A819C018091B7039091B803F901E80F04
:101C9000F91F8985808389819A8101969A83898336
:101CA0008B819C8101979C838B838B819C812FEFFF
:101CB0008F3F920791F189819A819C018091B703AE
:101CC0009091B803F901E80FF91F8F818083898112
:101CD0009A8101969A8389838B819C8101979C8349
:101CE0008B838B819C812FEF8F3F9207B1F089818D
:101CF0009A819C018091B7039091B803F901E80F94
:101D0000F91F8D81808389819A8101969A838983C5
:101D10008B819C81009709F02CCF64960FB6F894C4
:101D2000DEBF0FBECDBFDF91CF910895CF93DF937C
:101D3000CDB7DEB7E9E2F0E082E28083E0E4F0E0F4
:101D40001082E0E2F0E082E28083ECE5F0E01082D5
:101D5000A2E3B0E0E2E3F0E0808181608C93A8E34D
:101D6000B0E0E8E3F0E0808184608C93EAE2F0E0A8
:101D700088E98083E0E4F0E086E88083EBE2F0E04D
:101D800082EC8083E1E2F0E088E98083ECE5F0E03A
:101D900086E88083E2E2F0E082EC8083DF91CF91FD
:101DA0000895CF93DF93CDB7DEB721970FB6F894A0
:101DB000DEBF0FBECDBF8983EBE2F0E080819927C3
:101DC000807290700097C1F3ECE2F0E0898180832B
:101DD00021960FB6F894DEBF0FBECDBFDF91CF9135
:101DE0000895CF93DF93CDB7DEB726970FB6F8945B
:101DF000DEBF0FBECDBF9E838D838D819E81DC01B2
:101E0000FD0101900020E9F73197CF018A1B9B0B60
:101E10009C838B831A8219820FC029813A818D811C
:101E20009E81F901E80FF91F80810E94D10E8981FE
:101E30009A8101969A83898329813A818B819C8139
:101E40008217930750F78091B9030E94D10E8091B9
:101E5000BA030E94D10E26960FB6F894DEBF0FBECD
:101E6000CDBFDF91CF910895CF93DF93CDB7DEB78C
:101E700066970FB6F894DEBF0FBECDBF9E8B8D8BDD
:101E80008D899E894AE050E09E012F5F3F4FB90146
:101E90000E94BA11CE0101960E94F10E66960FB60D
:101EA000F894DEBF0FBECDBFDF91CF910895CF93E1
:101EB000DF93CDB7DEB722970FB6F894DEBF0FBE23
:101EC000CDBF8A8387E089831FC08A81482F552729
:101ED0008981282F332727FD309581E090E0022E5D
:101EE00002C0880F991F0A94E2F7842395231816DD
:101EF000190624F481E30E94D10E03C080E30E94FE
:101F0000D10E89818150898389818823F4F680915B
:101F1000B9030E94D10E8091BA030E94D10E22967D
:101F20000FB6F894DEBF0FBECDBFDF91CF910895FD
:101F30001F920F920FB60F9211242F933F938F93FE
:101F40009F93AF93BF93EF93FF93CF93DF93CDB75F
:101F5000DEB72297DEBFCDBFE3E2F0E08081809361
:101F6000A8048091A8048D30D1F48091CA038130F7
:101F7000B1F4A5E3B0E0E5E3F0E08081877F8C93E6
:101F80001092CA0381E08093CB0380916204992769
:101F90002091A804FC01E453FC4F208348C08091A9
:101FA000CA03282F33273A83298389819A8100978E
:101FB00031F029813A812130310521F138C08091F9
:101FC000A804833271F48091CB03882351F481E01B
:101FD0008093CA03A5E3B0E0E5E3F0E08081886088
:101FE0008C931092620430916204832F9927209180
:101FF000A804FC01E453FC4F2083832F8F5F809360
:10200000620415C08091620499272091A804FC0104
:10201000E453FC4F208380916204863930F4809130
:1020200062048F5F8093620402C01092CA032296FA
:10203000F894DEBFCDBFDF91CF91FF91EF91BF91BB
:10204000AF919F918F913F912F910F900FBE0F9065
:102050001F901895CF93DF93CDB7DEB76E970FB66D
:10206000F894DEBF0FBECDBF2091680430916904A3
:10207000CE010B964AE050E0BC01C9010E94BA11A2
:1020800080E4898384E48A8380E38B831C82CE018D
:102090000B96DC01FD0101900020E9F73197CF019B
:1020A0008A1B9B0B9E01255F3F4FAC01B901CE01FE
:1020B00001960E94AA11CE010196DC01FD0101905A
:1020C0000020E9F731979F012A1B3B0BCE010196B7
:1020D000820F931FFC0183E290E091838083CE0105
:1020E00001960E94F10E20916A0430916B04CE019A
:1020F0000B964AE050E0BC01C9010E94BA1180E48D
:10210000898384E48A8381E38B831C82CE010B96CE
:10211000DC01FD0101900020E9F73197CF018A1B16
:102120009B0B9E01255F3F4FAC01B901CE0101968B
:102130000E94AA11CE010196DC01FD010190002050
:10214000E9F731979F012A1B3B0BCE010196820FC5
:10215000931FFC0183E290E091838083CE0101967E
:102160000E94F10E2091720430917304CE010B96FF
:102170004AE050E0BC01C9010E94BA1180E48983A1
:1021800088E68A838DE38B831C82CE010B96DC016B
:10219000FD0101900020E9F73197CF018A1B9B0BCD
:1021A0009E01255F3F4FAC01B901CE0101960E940F
:1021B000AA11CE010196DC01FD0101900020E9F792
:1021C00031979F012A1B3B0BCE010196820F931F73
:1021D000FC0183E290E091838083CE0101960E940E
:1021E000F10E20917A0430917B04CE010B964AE0E7
:1021F00050E0BC01C9010E94BA1180E4898386E5E0
:102200008A838CE68B831C82CE010B96DC01FD0158
:1022100001900020E9F73197CF018A1B9B0B9E01AB
:10222000255F3F4FAC01B901CE0101960E94AA1172
:10223000CE010196DC01FD0101900020E9F7319704
:102240009F012A1B3B0BCE010196820F931FFC01BD
:1022500083E290E091838083CE0101960E94F10E8B
:102260002091C4033091C503CE010B964AE050E0A3
:10227000BC01C9010E94BA1180E4898386E58A8382
:1022800081E48B831C82CE010B96DC01FD01019061
:102290000020E9F73197CF018A1B9B0B9E01255F38
:1022A0003F4FAC01B901CE0101960E94AA11CE01A7
:1022B0000196DC01FD0101900020E9F731979F01B3
:1022C0002A1B3B0BCE010196820F931FFC0183E278
:1022D00090E091838083CE0101960E94F10E6E966C
:1022E0000FB6F894DEBF0FBECDBFDF91CF9108953A
:1022F000CF93DF93CDB7DEB7A5E3B0E0E5E3F0E041
:10230000908182E089278C93DF91CF910895CF93BC
:10231000DF93CDB7DEB78091C3038130C1F48091E4
:10232000C203813051F4A5E3B0E0E5E3F0E0808141
:102330008E7F8C931092C2030AC0A5E3B0E0E5E360
:10234000F0E0808181608C9381E08093C203DF9113
:10235000CF910895FB01DC010D900020E9F7119762
:102360004150504028F0019000200D92C9F7089587
:102370001C920895FB019F01E8944230C4F045325D
:10238000B4F44A3029F497FB1EF4909581959F4F41
:10239000642F77270E94FE11805D8A330CF0895DDF
:1023A0008193CB010097A1F716F45DE2519310825F
:1023B000C9010C94DB11DC01FC0101900020E9F75C
:1023C0003297AE17BF0730F47C91608170833197EC
:1023D0006D93F7CF089597FB092E07260AD077FD56
:1023E00004D00CD006D000201AF4709561957F4F70
:1023F0000895F6F7909581959F4F0895AA1BBB1BF2
:1024000051E107C0AA1FBB1FA617B70710F0A61BF4
:10241000B70B881F991F5A95A9F780959095BC0115
:04242000CD0108954D
:1024240001125A2C294400000A31002300230054CD
:1024340064665363655262005161005060005060ED
:1024440000516100526200536365546466676869B1
:102454006A6B6B6A696867955550A55540A5550028
:10246400A55500A95500AAAAAAAAAAAAAAAAAAAACC
:10247400AAAAAAAA94AAA940AA9550AA5554AA55A8
:1024840055AA5555AA5555AA5555AA0155555555F8
:102494005555555555555500005600001500000575
:1024A400000005000005A80001A80001A8000550CF
:1024B40000050000050000150000550001554015F9
:1024C40055555555556AAA556AAA55AAAA5555553A
:1024D40055555555555555AAAAAA6AAAAA5AAAAA3B
:1024E40056AAAA56AAAA56AAAA56AAAA56AAAA5640
:1024F400AAAA56AAAA56AAAA56AAAA56AAAA56AADC
:10250400AA56AAAAAAAAAAAAAAAAAAAAAA5555557A
:1025140055555555555555956A55956A55A56A9518
:10252400A56A95A55A95A55A95A55A95A55A95A50E
:102534005A95A55A95A55A95A55A95A55A95A55A59
:1025440095A56A95A56A95956A55956A5555555503
:102554005555555555555555A95655AA56556A5567
:10256400556A55556A55556A95555A95555AA555FE
:1025740056A55556A55556A95555AA55556A5555A6
:102584006A55555A55555A555556555555555555D7
:1025940055555555555555AAAAAAAAAAAAAAAAAAEA
:1025A400AAAAAAAAAAAA6AAAAA6AAAAA5AAAAA5AA7
:1025B400AAAA56AAAA56AAAA55AAAA556AAA956A5E
:1025C400AA955AAAA556AAA955AAAA556A5555550F
:1025D40055555555555555A95400AA9555AAA9556B
:1025E400AAAA95AAAAA5AAAAAAAAAAAAAAAAAAAA61
:1025F400AAAAAAAAAAAAAAAAAAAAAAAAAAAAAAAA37
:10260400AAAAA9AAAAA96AAAA96AAAA569555555EE
:1026140055555555555555555541555541555500E3
:10262400555500555400555400A55400AA5400AA09
:10263400A500AAA500AAA540AAA550AAA554AAA582
:1026440055AAA555AAA555AAA5556AA555555555E2
:1026540055555555555555AA0055AA0015AA0015A6
:102664006A00052A00052A0005000005000005008F
:10267400000600001600001A00005A00056A5555AD
:102684006A5555AA5555AA5556AA555AA955555588
:102694005555555555555555AAAA56AAAA56AAAAE6
:1026A4005AAAAA5AAAAA6AAAAA6AAAAAAAAAAAAAA6
:1026B400AAAAAAAAAAAAAAAAAAAAAAAAAAAAAAAA76
:1026C400AAAAAAAAA96AAAA96AAA5A5AAA55555587
:0C26D4005555555555555566040D0A0026
:00000001FF
